:100000003FC059C058C057C056C055C054C053C057
:1000100052C002C250C04FC04EC04DC04CC04BC0B9
:100020004AC049C048C00000000037003400310019
:1000300000000000380035003200000000003600EB
:100040003300300004040404040404040202020225
:10005000020203030303030301020408102040808B
:100060000102040810200102040810200000000012
:100070000000000000030405000000000000000074
:1000800011241FBECFE5D4E0DEBFCDBF10E0A0E657
:10009000B0E0EEE1F7E002C005900D92A236B107A4
:1000A000D9F710E0A2E6B0E001C01D92AE36B1076C
:1000B000E1F727D332C3A4CF8CE0E9D2892B69F4CE
:1000C00082E1E5D2019749F481E160E0A7D282E1C3
:1000D00060E0A4D281E0809362008BE0D8D2892BCB
:1000E00069F481E1D4D2019749F481E160E096D2CC
:1000F00082E160E093D281E0809362000895809174
:100100006000909161008230910549F18330910542
:1001100034F4009779F0019709F089C01DC084304C
:10012000910509F44BC08430910564F1059709F0FD
:100130007EC063C080E161E071D282E160E06ED296
:1001400083E160E06BD281E160E068D289E09FD218
:10015000019709F06CC047C082E090E049C061E0BF
:1001600070E080E090E0A0D180E161E057D282E1D0
:1001700060E054D283E160E051D281E161E04ED28F
:100180008BE02EC061E070E080E090E08DD180E1F6
:1001900060E044D282E160E041D283E161E03ED29E
:1001A00081E160E03BD289E072D2892B09F03FC047
:1001B00068EE73E080E090E077D115C061E070E018
:1001C00080E090E071D180E160E028D282E161E0DE
:1001D00025D283E160E022D281E160E01FD28CE091
:1001E00056D2892B21F58091600090916100019693
:1001F0009093610080936000089561E070E080E07A
:1002000090E052D180E161E009D282E160E006D263
:1002100083E160E003D281E160E000D28091600080
:100220009091610001969093610080936000089521
:1002300080916000909161000697A1F488E027D238
:10024000892B31F483E161E0E9D180E160E0E6D11E
:1002500087E01DD2892B31F483E160E0DFD180E1BA
:1002600061E0DCD180E013D2892B09F047C0809196
:10027000630090916400019709F040C01092610002
:100280001092600010926400109263000AC0809186
:10029000630090916400892B29F4309364002093CB
:1002A00063002DDF81E0F3D1892B79F58091630024
:1002B00090916400019749F580E160E0AFD182E15F
:1002C00060E0ACD183E160E0A9D181E160E0A6D13A
:1002D00085E090E09093610080936000109264004C
:1002E0001092630008958091630090916400892BBF
:1002F00091F43093640020936300089580E0C7D1A7
:100300009C018130910571F6C2CF81E0C0D19C0182
:100310008130910541F308958BDFCEDEF0DE089544
:1003200080E161E03CD180E160E078D181E161E091
:1003300036D181E160E072D182E161E030D182E1C9
:1003400060E06CD183E161E02AD183E160E066D1B5
:1003500087E060E024D187E061E060D188E060E080
:100360001ED188E061E05AD186E060E018D186E0D5
:1003700061E054D185E060E012D185E061E04ED1CA
:1003800080E060E00CD180E061E048D181E060E095
:1003900006D181E061E042D18BE060E000D18BE0EA
:1003A00061E03CD18CE060E0FAD08CE061E036D1D5
:1003B0008AE060E0F4D08AE061E030D189E060E07A
:1003C000EED089E061E02AD164EF71E080E090E056
:1003D0006BD080E161E022D182E160E01FD183E156
:1003E00060E01CD181E160E019D164EF71E080E050
:1003F00090E05AD080E160E011D182E160E00ED15E
:1004000083E160E00BD181E160E008D164EF71E04D
:1004100080E090E049D008951F920F920FB60F929E
:1004200011242F933F938F939F93AF93BF9380910A
:10043000690090916A00A0916B00B0916C003091BE
:100440006D000196A11DB11D232F2D5F2D3720F0CA
:100450002D570196A11DB11D20936D008093690059
:1004600090936A00A0936B00B0936C00809165003C
:1004700090916600A0916700B09168000196A11D5F
:10048000B11D8093650090936600A0936700B093C0
:100490006800BF91AF919F918F913F912F910F90E5
:1004A0000FBE0F901F9018959B01AC017FB7F89479
:1004B0008091650090916600A0916700B0916800FE
:1004C00062B708B600FE05C06F3F19F00196A11D86
:1004D000B11D7FBFBA2FA92F982F8827860F911D96
:1004E000A11DB11D62E0880F991FAA1FBB1F6A954D
:1004F000D1F7BC012EC0FFB7F894809165009091B0
:100500006600A0916700B0916800E2B708B600FEEF
:1005100005C0EF3F19F00196A11DB11DFFBFBA2F15
:10052000A92F982F88278E0F911DA11DB11DE2E0E4
:10053000880F991FAA1FBB1FEA95D1F7861B970B3F
:10054000885E9340C0F22150304040405040685196
:100550007C4F211531054105510569F608957894C0
:1005600083B7826083BF83B7816083BF89B78160AF
:1005700089BF1EBC8EB582608EBD8EB581608EBD7A
:100580008FB581608FBD85B5846085BD85B580647C
:1005900085BD329A319A309A379A1AB80895CF9316
:1005A000DF93482F50E0CA01885A9F4FFC013491D5
:1005B0004C5B5F4FFA018491882369F190E0880FCA
:1005C000991FFC01EA5DFF4FA591B491FC01E05D2C
:1005D000FF4FC591D491662351F42FB7F8948C91B5
:1005E000932F909589238C93888189230BC0623047
:1005F00061F42FB7F8948C91932F909589238C9365
:100600008881832B88832FBF06C09FB7F8948C9175
:10061000832B8C939FBFDF91CF910895482F50E09B
:10062000CA0184599F4FFC012491CA01885A9F4FE7
:10063000FC0194914C5B5F4FFA013491332331F10B
:10064000222381F0243039F0253049F0233051F451
:100650008FB58F7702C08FB58F7D8FBD03C085B5F5
:100660008F7D85BDE32FF0E0EE0FFF1FE05DFF4FB4
:10067000A591B4912FB7F894662321F48C919095AD
:10068000892302C08C91892B8C932FBF0895682FEA
:1006900070E0CB0184599F4FFC012491CB01885A13
:1006A0009F4FFC0144916C5B7F4FFB019491992318
:1006B00019F420E030E022C0222381F0243039F008
:1006C000253049F0233051F48FB58F7702C08FB5B4
:1006D0008F7D8FBD03C085B58F7D85BD892F90E04F
:1006E000880F991F865C9F4FFC01A591B4918C9156
:1006F00020E030E0842311F021E030E0C9010895CA
:100700000895CF93DF932BDFFBDF0ADEC0E0D0E05C
:0E07100003DE2097E9F374DCFBCFF894FFCFF3
:02071E000600D3
:00000001FF
